:020000040000FA
:1000000083160313810180298B138B1B042897000F
:10001000030E980083010A0899008A0183130408DB
:100020009A009408031D1728051A33283628140847
:10003000083C031C2328051E9513051A9517031960
:100040003628950C36281408093C031C2828362825
:10005000051E33281017831603130610831203138B
:1000600006100B123428950194013728940A8B103E
:100070001A08840019088A00180E8300970E170EBC
:10008000090015089600F03C031D492810141011B2
:100090003529101C902810101508123C03195328FC
:1000A0001508593C031990101508583C031D5E288B
:1000B000901D5C2890113529901535291508113CA3
:1000C000031D6428101243291508143C031D35290B
:0400D000901243291E
:10012000101D9E2815084A3C031D99282F30950064
:10013000CE2815085A3C03189E2835291508613C1D
:100140000318B4280E3095021508613C031CAB2837
:1001500019309507B4281508773C0318B4281508FA
:10016000D23C03191015352903308A001508612384
:1001700095009508031935291508603C0318442992
:1001800015087A3C031C442915089019CA28901CAC
:10019000CE28CC289018CE28E03E950015089B006C
:1001A00057221B087A3C031C35291B08403C0318C6
:1001B000E2289B121B08403C031835291B0D923E78
:1001C0009E0025291B082F3C0318EE281B08393CEC
:1001D000031C18291B0D9F3E9E0025291B08223C4D
:1001E000031DF428483023291B08273C031DFA2847
:1001F0004A3023291B08283C031D00294C302329A1
:100200001B08293C031D06294C3023291B082C3CC4
:10021000031D0C294E3023291B082D3C031D1229D8
:10022000503023291B082E3C031D35295230232929
:100230001B083A3C031D1E29543023291B083F3C50
:10024000031D352956309E00252990179E00033046
:100250008A001E080723A1009E0A1E080723A0008B
:1002600035290D3057220A3008008316031306146F
:100270008312031310130B16080090140034101689
:100280000034901600343529901CCE2815080D3CFA
:100290000318CE281608613C031CCE2816083C3CE7
:1002A000031855293D3096025E291608243C031890
:1002B0005C29233096025E290430960703308A00B9
:0802C0001608DA239500CE2890
:1003000005100511851183120313051405118316B9
:100310000313061405160113831203130B1694011D
:100320009001F8308B058B172A308E0002308A003E
:100330000E082A3CD02257228E0B9629FF308C00C3
:100340000230852290308C0003308522C0308C0032
:0E03500003308522101B4120901BB021AA29EA
:100360002008A2002108A30090139F0102309B00E7
:1003700008309C009B1823089B1C22089D009D1F91
:10038000C3299F0ADA299F080319DA2905151F08CE
:10039000013C031CD02991308C0001308522D429E6
:1003A000FA308C00053085220511063040220630D7
:1003B0004E229F019D0D9C0BBF299B0BB829083035
:0803C000402206304E22080025
:100480008C00810183160313C030810508008C00A5
:10049000810183160313C03081050130810483126A
:1004A00003130B110B1D522A8C0B512A08009200CA
:1004B000051008308C00682212180514121C051053
:1004C000920C68228C0B5C2A0514682268220800B2
:1004D0001D308D006E2A0B308D006E2A8D0B6E2A1A
:1004E00008006B220618832A08308C006822061840
:1004F0009317061C93130C0B930C8C0B762A682213
:10050000061C93010800930138288D008101831691
:10051000031307308100831203130B1185159722F3
:10052000851197220B1D8E2A8D0B8D2A08000C0831
:080530008E008E0B992A0800D1
:1005A00082075034493443342034313436344634AD
:1005B0003834343420344134543420344B346534AA
:1005C000793462346F3461347234643420344434A6
:1005D000653463346F346434653472342034633486
:1005E0006F346E346E34653463347434653464341B
:0605F0000D340A340A3448
:02060E00820761
:10061000DB346C34B634D834AD34B034AB346034FD
:10062000AA34C034AA348034D5344034DA34A03407
:10063000DB345034DB346834B0340034D534003427
:10064000D6348034D434003480340034AD340034B3
:10065000DA340034AA340034A0340034B634C03460
:10066000D6340034B5340034D8340034D0340034B7
:10067000DB340034B6348034DA34C034B43400347B
:10068000A8340034C0340034AC340034AB3400340B
:10069000B6340034D5348034D634C034DA348034BF
:1006A000B5346834B634DA34D634D634DA34B634C1
:1006B000D5345834B534AC34DB345434AD34A83488
:0E06C200820700343934003435343334313497
:1006D000323432340034303438343634343409343B
:1006E0007E34003400343F293D29003441297134DF
:1006F00031340034003400347A3473346134773464
:10070000323400340034633478346434653434343F
:100710003334003400342034763466347434723424
:100720003534003400346E346234683467347934DC
:1007300036340034003400346D346A347534373460
:100740003834003400342C346B3469346F34303432
:100750003934003400342E343F346C343B3470343C
:100760002D34003400340034273400345B342B340F
:100770000034003400343D2931295D3400347C34A8
:100780000034003400343C3430342E3432343534C8
:10079000363438340034003431342B3433342D348F
:1007A0002A343934003408340034003431343734D6
:1007B00034343734820726342A34243423343C3406
:1007C00000340034003429342834003425343E34D5
:1007D0002F3400343A3400345F3460345E340034F3
:1007E000223400347B343D3400342134003400346E
:1007F00000347D3400345C340034403400343E3402
:02400E00F13F80
:00000001FF
